:0200000480007A
:10000000971F0000938F0F00171100001301810349
:1000100083C10F0003C21F0083C22F0003C33F0030
:100020002320310023224100232451002326610094
:10003000171C0000130C5CFD9712000093828201D4
:10004000834CFCFF034D0C00834D1C00034E2C0021
:1000500023A0920123A2A20123A4B20123A6C201DC
:1000600097130000938373FA17140000130484FF9E
:1000700003CF130083CF230083C0330003C14300A9
:100080002320E4012322F401232414002326240046
:10009000171500001305C57797150000938585FD9A
:1000A00003460580834615800347258083473580B6
:1000B00023A0C50023A2D50023A4E50023A6F500B4
:1000C000970600009386467517170000130787FBF5
:1000D00083C7C67F03C8D67F83C8E67F03C9F67F80
:1000E0002320F700232207012324170123262701B9
:1000F00017180000130888F297180000938888F9F1
:100100000349C8FF8349D8FF034AE8FF834AF8FF41
:10011000034B0800834B1800034C2800834C380025
:10012000034D4800834D5800034E6800834E78000D
:1001300023A0280123A2380123A4480123A65801A3
:1001400023A8680123AA780123AC880123AE980173
:1001500023A0A80323A2B80323A4C80323A6D8037B
:10016000971A0000938A0AEC171B0000130B8BF5FB
:1001700003C00A0023200B00971A0000938ACAEAE2
:10018000171B0000130B4BF483AB0A0003CC0B00CE
:10019000930C0C0023209B01971C0000938C4CE9CE
:1001A000171D0000130D8DF283CC0C0023209D0140
:1001B000971D0000938D1DE8171E0000130E4EF1D1
:1001C00083CDFDFF2320BE0117150000130585E731
:1001D00097150000938505F0370610F01306C6F258
:1001E0006306B5028326C5002320D600832685003A
:1001F0002320D600832645002320D6008326050031
:100200002320D600130505016FF09FFD370510F080
:10021000130505F223200500000000000000000087
:0402200000000000DA
:1010000022F2F111F44433F366F6F555F88877F7D8
:10101000AA0A09990CCCBB0BEE0E0DDDF000FF0FF8
:101020007856341228100080F0DEBC9A10325476C4
:1010300098BADCFE00000000000000000000000084
:10104000FFFFFFFFFFFFFFFFFFFFFFFFFFFFFFFFB0
:10105000FFFFFFFFFFFFFFFFFFFFFFFFFFFFFFFFA0
:10106000FFFFFFFFFFFFFFFFFFFFFFFFFFFFFFFF90
:10107000FFFFFFFFFFFFFFFFFFFFFFFFFFFFFFFF80
:10108000FFFFFFFFFFFFFFFFFFFFFFFFFFFFFFFF70
:10109000FFFFFFFFFFFFFFFFFFFFFFFFFFFFFFFF60
:1010A000FFFFFFFFFFFFFFFFFFFFFFFFFFFFFFFF50
:1010B000FFFFFFFFFFFFFFFFFFFFFFFFFFFFFFFF40
:1010C000FFFFFFFFFFFFFFFFFFFFFFFFFFFFFFFF30
:040000058000000077
:00000001FF
